:100000000C945D000C94CA010C947A000C947A0054
:100010000C947A000C947A000C947A000C947A0078
:100020000C947A000C947A000C947A000C947A0068
:100030000C947A000C947A000C947A000C947A0058
:100040000C947A000C947A000C947A000C947A0048
:100050000C947A000C947A000C947A000C947A0038
:100060000C947A000C947A000902120001010080BD
:100070001909040000000000000012011001FF0037
:100080000008C016DC050401010200010E03550042
:10009000530042006100730070001C03770077007A
:1000A00077002E00660069007300630068006C0032
:1000B0002E00640065000403090411241FBECFEF65
:1000C000D8E0DEBFCDBF11E0A0E0B1E0E6E2F2E1B2
:1000D00002C005900D92A230B107D9F711E0A2E05D
:1000E000B1E001C01D92AC34B107E1F70E94FF08F6
:1000F0000C9411090C940000CF93DF9360912801B8
:10010000635067FD13C080912501CCE0D0E0C81B8F
:10011000D109C45DDE4F809124018D3209F458C0AD
:100120008091020187FD9DC01092280180910001FD
:1001300084FF41C0609101016F3F09F43CC0693008
:1001400008F470C06850609301018091180198E82C
:1001500089278093180168E08091020187FD1DC006
:10016000409126015091270186FF72C0FA01862F27
:10017000A9E1B1E094919D9331968150D9F7262F52
:10018000215030E02F5F3F4F240F351F3093270160
:1001900020932601C62FCC5F50C089E191E00E94D8
:1001A000BF07682F893008F4A4C08FEF8093010146
:1001B000CEE1C093000194E183B1837031F491509A
:1001C000D9F71092290110922301DF91CF91089560
:1001D000683009F0A9CF83EC809318018AE58093F9
:1001E0000001109202018881807609F045C09A8151
:1001F00010922101898181114AC01092220121E2CD
:1002000031E082E030932701209326018F3FC1F136
:100210009F81911104C09E81981708F4892F8093C3
:10022000010182CF109201018091180198E889277D
:1002300080931801611190CFC4E089E191E00E94A0
:10024000C601CC3009F4B5CF8FEF80930101B1CF57
:10025000DA01862FE9E1F1E09D9191938150E1F778
:100260008ECFCE010E942F088F3FF9F0882309F42A
:100270005BCF1092010158CFCE010E940B06C6CF72
:10028000988197FD16C090E890930201C8CF853001
:1002900091F0863001F18830D1F0893091F021E27F
:1002A00031E08A3021F180E0ADCF8EE18093000112
:1002B0003BCF8E81E8CF9093290121E231E080E0AD
:1002C000A1CF90932B0121E231E080E09BCF2BE284
:1002D00031E081E097CF8B81813001F18230B1F044
:1002E000833051F080E090E4909302018FCF81E061
:1002F00089CFC82FCC5FA1CF911118C086EB90E0B9
:10030000909327018093260184E0EDCF88E690E06A
:10031000909327018093260182E1E5CF8AE790E060
:10032000909327018093260182E1DDCF913051F037
:100330009230C1F68CE890E09093270180932601DB
:100340008EE0D1CF8AE990E0909327018093260137
:100350008CE1C9CFE9E6F0E0808183608083E89A90
:100360000895A82FB92F80E090E041E050EA609511
:1003700030E009C02D9182279795879510F084274A
:100380009527305EC8F36F5FA8F30895EADF8D9379
:100390009D930895CF93CFB7CF93DF93C395189BC9
:1003A000E9F7189B0BC0189B09C0189B07C0189B46
:1003B00005C0189B03C0189B01C089C06F93C091F2
:1003C0002501DD27C45DDE4F2F9365E5189B03C033
:1003D0002F916F91E6CF0F931F934F9320E040E151
:1003E0005F9303B1037000FB27F93F9350E03BE0BC
:1003F00039C0137040642F77012F5F5F1EC04068C3
:1004000013B113702F7752501FC0406403B12F7780
:100410000370D1F15F5F00C023C0406213B12F773A
:10042000137091F15F5F00C025C003701027515019
:1004300012F45D5F0000115027952C3F13B1C8F6F0
:1004400013700127015027952C3FC8F64227499386
:1004500003B1037010274F73115027952C3FA8F656
:100460004695469513B1137079F0012701502795F1
:100470002C3F98F66B5A60F3315003B1B0F600C0D0
:1004800011E01CBB002717C03B503195C31BD04067
:1004900011E01CBB0881033CF9F00B34E9F020911A
:1004A00023011981110F1213EDCF093651F10D32CD
:1004B00011F0013E39F700932A013F915F914F916E
:1004C0001F910F912F916F91CCB3C0FD67CFDF913A
:1004D000CF91CFBFCF91189520912A01222369F3A4
:1004E00010912801112339F534303AF13093280165
:1004F00020932401109125013BE0311B309325010D
:100500001CC0009128010130B4F40AE530910001CB
:1005100034FD14C000930001C8E1D1E013C00527E9
:1005200010E000C0000005B91AC0052710E0221F26
:100530001DC010E021C04AE502C032ED432FC4E1E6
:10054000D0E032E014B11360289A05B114B953E039
:1005500020E865E320FF052705B9279517951C3F7F
:10056000F0F66695B8F7B1F720FF052705B927958E
:1005700017951C3FD0F62795179517FF0527000004
:100580001C3F05B9B0F629913A9519F70C7F1091E7
:100590002901110FC651D04005B911F01093230164
:1005A00011E01CBB016014B11C7F402F4C7F54E054
:1005B0005A95F1F705B914B945B97FCF682F58E0BE
:1005C00080E0709148012091470167FD1EC02B9883
:1005D000660F880F1C998F5F2D9A36B5472F4150B3
:1005E00030F096B5931B9217E0F34150D0F72D9859
:1005F00036B5472F415030F096B5931B9217E0F374
:100600004150D0F7515009F708952B9AE1CF8EBD94
:100610000DB407FEFDCF8EB5089521E1969587951F
:10062000779567952A95D1F7209146012617D9F03D
:1006300060934601E0914301F09144018DE40995F6
:10064000E0914301F091440180E00995E09143017C
:10065000F0914401809146010995E0914301F091A8
:10066000440180E009940895809145018CBD8091FA
:1006700042018DBD08958823B1F0893008F04AC049
:100680002EED32E0309344012093430191E09093AA
:100690004801853001F1C0F08730A1F168F588E0AC
:1006A00080934701089587E093E0909344018093FD
:1006B00043011092420181E08093470180934801F9
:1006C00082E5809345010895833001F140F080E296
:1006D00080934701089580E1809347010895823017
:1006E00039F080E88093470182E0809348010895C3
:1006F00080E8809347010895883099F782E08093DD
:100700004701089584E080934701089580E4809331
:100710004701089527E033E03093440120934301DB
:100720001092420191E090934701909348018930E3
:1007300049F030F28B3051F08C3011F681E5809326
:100740004501089583E580934501089582E58093EE
:10075000450190934201089526B53091480190914A
:100760004701315030F086B5821B8917E0F33150D4
:10077000D0F7089584B18C6284B92A982D9826B553
:1007800030914801432F90914701415030F086B598
:10079000821B8917E0F34150D0F72A9A26B53150D1
:1007A00030F086B5821B8917E0F33150D0F72A98D4
:1007B00080914301909144018750934019F0109229
:1007C00046010895809145018CBD809142018DBD07
:1007D00010924601089584B1837D84B985B1837DEB
:1007E00085B91CBC0895CF93DF93C0E2E09143012B
:1007F000F09144018CEA0995E0914301F0914401A4
:1008000083E50995E0914301F091440180E0099569
:10081000D82FE0914301F091440180E00995D33550
:1008200009F43AC01CBC26B530914801432F909181
:100830004701415030F086B5821B8917E0F34150E3
:10084000D0F72A9A26B5432F415030F086B5821B47
:100850008917E0F34150D0F72A9826B5315030F08F
:1008600086B5821B8917E0F33150D0F7E091430140
:10087000F091440183E0E730F80739F0C15009F006
:10088000B9CF81E0DF91CF910895809145018CBD72
:10089000809142018DBDF2CF80E0DF91CF9108952C
:1008A000CF92DF92EF92FF926B017C010E940D03C9
:1008B000D701C60181709927AA27BB27880F880F07
:1008C000880FE0914301F091440180620995D701BE
:1008D000C60139E0B695A795979587953A95D1F7D2
:1008E000E0914301F09144010995D701C601B69505
:1008F000A79597958795E0914301F091440109955B
:10090000E0914301F091440180E0FF90EF90DF908F
:10091000CF900994CF92DF92EF92FF920F931F93A3
:10092000CF93DF936B017C01C42FD22F0E940D0364
:10093000970186010170112722273327802F880F06
:10094000880F880FE0914301F0914401806409957C
:10095000D701C60159E0B695A795979587955A9501
:10096000D1F7E0914301F09144010995D701C60107
:10097000B695A79597958795E0914301F09144012D
:100980000995E0914301F09144018C2F0995DD23F5
:10099000B9F0CF3791F0D6B5CEE1C701B6010E94CC
:1009A00050048F3769F486B58D1B813510F0D6B5AC
:1009B000C150C111F2CF81E004C08FE00E949605C2
:1009C00080E0DF91CF911F910F91FF90EF90DF902A
:1009D000CF900895CF92DF92EF92FF920F931F93E3
:1009E000CF93DF931F92CDB7DEB76B017C014983B4
:1009F0000E940D03E0914301F09144018CE40995BC
:100A0000D701C60179E0B695A795979587957A9510
:100A1000D1F7E0914301F09144010995D701C60156
:100A2000B695A79597958795E0914301F09144017C
:100A30000995E0914301F091440180E009954981D5
:100A40004F3FE9F006B51EE1C701B6010E94500410
:100A50008F3F99F486B5801B813510F006B5115093
:100A60001111F2CF81E00F90DF91CF911F910F9183
:100A7000FF90EF90DF90CF90089580E0F4CF8FE06B
:100A80000E94960580E0EFCF1F93CF93DF931F92D4
:100A9000CDB7DEB7182FE0914301F091440180EA11
:100AA00099830995E0914301F09144019981892F3F
:100AB0000995E0914301F0914401812F0995E0915E
:100AC0004301F091440180E00F90DF91CF911F919D
:100AD00009941F93CF93DF9300D0CDB7DEB7182FC3
:100AE000E0914301F091440180EC6A839983099578
:100AF000E0914301F09144019981892F0995E0919A
:100B00004301F0914401812F0995E0914301F09157
:100B100044016A81862F09958EE10E94960580E046
:100B20000F900F90DF91CF911F910895882349F086
:100B300030E026B596B5921B9035E0F33F5F381351
:100B4000F8CF0895259A23982B9A50E217D05A95FA
:100B5000E9F70895AC0188E605D0842F03D089E633
:100B600001D0852F0FD028E030E0382780FB869514
:100B700006D02A95D1F730FB02D000D06894239894
:100B80002B9A16F02B98239AE0914A01F0914B0191
:100B90003197F0F72D9AE3B1E3FBE0914A01F09130
:100BA0004B013197F0F72D98089520ECE7DF46F4DC
:100BB0002A95E1F780E02AE1E5DF2A95E9F7DECF23
:100BC00028E030E0DBDF869587F938272A95D1F7D2
:100BD000D5DF27F9322772F3D1DFD0CFDB01742FB5
:100BE000B9DF84E2BFDFE1DF8D937A95D1F7089515
:100BF000DB01742FAFDF83EFB5DF8DE1B3DF84E678
:100C0000B1DF8D91AFDF82E7ADDFCFDF8078D9F73D
:100C10007A9589F70895CF93DF93EC01898181302C
:100C200089F1823009F4ABC0833009F461C08430AB
:100C3000B1F1873009F482C0853009F402C18630F1
:100C400009F4A2C0883009F4D5C0893009F4FFC086
:100C50008A3009F42AC18B3009F456C18C3009F46A
:100C600069C18D3009F480C18E3009F483C18F30A1
:100C700009F4FEC0803109F41FC18F3709F439C16E
:100C800080E02DC0329B56C0809103010E943B033F
:100C90001092040141980E94BA0380E020C0809124
:100CA0000401811110C05B8140E08A81482B6627D6
:100CB00057FD6095762F40930D0150930E01609380
:100CC0000F01709310019F8180E02E81822B909301
:100CD00012018093110182E0809313018FEF25E0D0
:100CE00031E03093270120932601DF91CF910895C1
:100CF000E0914301F09144018A81099580930501B7
:100D0000E0914301F09144018B81099580930601A4
:100D1000E0914301F09144018C8109958093070192
:100D2000E0914301F09144018D8109958093080180
:100D300084E0D5CF85E00E943B03AACF80910401D7
:100D4000811110C05B8140E08A81482B662757FDE6
:100D50006095762F40930D0150930E0160930F0123
:100D6000709310019F8180E02E81822B909312015D
:100D70008093110183E0809313018FEFB0CF0E9425
:100D8000EB03419A80E0ABCF80910401811110C048
:100D90009B8180E02A81822BAA2797FDA095BA2FFC
:100DA00080930D0190930E01A0930F01B093100159
:100DB0003C812D81822F8F7080931601822F807F3E
:100DC00040E1849FC0011124830F911D9093150170
:100DD0008093140120FD809317019F8180E02E8174
:100DE000822B909312018093110181E08093130173
:100DF0008FEF75CF80910401811110C09B8180E03D
:100E00002A81822BAA2797FDA095BA2F80930D01E6
:100E100090930E01A0930F01B09310011092150151
:100E200010921401109216019F8180E02E81822B76
:100E3000909312018093110184E0809313018FEF4E
:100E40004ECF0E94F3038093050181E048CF81E0FB
:100E5000809304018A819B81AC81BD8180930D01C7
:100E600090930E01A0930F01B093100180E037CF53
:100E70009B8180E02A81822BAA2797FDA095BA2F1B
:100E800080930D0190930E01A0930F01B093100178
:100E90009F8180E02E81822B90931201809311011B
:100EA00085E0809313018FEF1ACF8A81809303012D
:100EB0001092050181E013CF9B8180E02A81822B73
:100EC000AA2797FDA095BA2F80930D0190930E014C
:100ED000A0930F01B09310019F8180E02E81822B9F
:100EE000909312018093110186E0809313018FEF9C
:100EF000F6CE81E080930501109206011092070161
:100F00001092080184E0EBCE9B8180E02A81822B45
:100F100090934B0180934A012A9A229A83E00E947F
:100F200096052A98419880E10E9496050E94A205A4
:100F300080E0D5CE80EC0E94B20580E00E94B20530
:100F40008AE00E9496052A9A85E00E9496052A98D2
:100F500085E00E94960584B1837D84B985B1837D47
:100F600085B9419A80E0BBCE0E94D50580930501EA
:100F700081E0B5CE8A810E94B20580E0B0CE0F93A9
:100F80001F93CF93DF93582F792F062F20911301B2
:100F9000322F3250323050F0253009F443C00FEF79
:100FA000802FDF91CF911F910F910895662391F1CA
:100FB00080910D0190910E01A0910F01B09110014F
:100FC000C52FD72F10E01CC00E9444058883809154
:100FD0000D0190910E01A0910F01B09110010196A9
:100FE000A11DB11D80930D0190930E01A0930F01DF
:100FF000B09310011F5F2196101751F0209113013B
:10100000223011F7BC01CD010E9450048883DFCF4C
:10101000083030F610921301802FDF91CF911F918D
:101020000F910895462F682F80910D0190910E0128
:101030000E94EE0580910D0190910E01A0910F018B
:10104000B0911001800F911DA11DB11D80930D0164
:1010500090930E01A0930F01B0931001A1CFFF92C6
:101060000F931F93CF93DF93382F792F162F209153
:101070001301213071F0243061F0263009F490C062
:10108000FF24FA948F2DDF91CF911F910F91FF9044
:101090000895112309F4B1C080910D0190910E01C2
:1010A000A0910F01B0911001C32FD72F00E0F12CB8
:1010B00050C02091140130911501232B09F053C029
:1010C00021E04881BC01CD010E948A0420911101D8
:1010D00030911201215031093093120120931101F6
:1010E000232BE9F4109213018091160181FF38C07F
:1010F0002091170130E0809114019091150128177B
:10110000390771F160910D0170910E0180910F010D
:101110009091100148810E94EA04FF24F394809189
:101120000D0190910E01A0910F01B0911001019657
:10113000A11DB11D80930D0190930E01A0930F018D
:10114000B09310010F5F2196011709F49BCF2091F6
:101150001301213009F4ADCF68810E946905B6CF33
:10116000FF24F394DCCF20E04881BC01CD010E9434
:101170008A04809117018150809317018111A6CFB5
:1011800060910D0170910E0180910F0190911001FD
:1011900048810E94EA04809114018093170196CF40
:1011A000462F682F80910D0190910E010E94F80545
:1011B00080910D0190910E01A0910F01B09110014D
:1011C000810F911DA11DB11D80930D0190930E0102
:1011D000A0930F01B0931001809111019091120121
:1011E000811B91099093120180931101892B29F49D
:1011F00010921301FF24F39445CFF12C43CF1BB879
:1012000015B88BEF8AB98FEF84B914B883E087B92A
:101210009EEF98B985BD0E94AA0178940E947C0037
:06122000FDCFF894FFCFA2
:021226005AFF6D
:00000001FF
